:100000000C9434000C9451000C9451000C94510049
:100010000C9451000C9451000C9451000C9451001C
:100020000C9451000C9451000C9451000C9451000C
:100030000C9451000C9451000C9451000C945100FC
:100040000C9453000C9451000C9451000C945100EA
:100050000C9451000C9451000C9451000C945100DC
:100060000C9451000C94510011241FBECFEFD4E02A
:10007000DEBFCDBF11E0A0E0B1E0EAE4FCE202C0E7
:1000800005900D92A038B107D9F711E0A0E8B1E0D2
:1000900001C01D92A438B107E1F70E9491000C94B1
:1000A00023160C9400001F920F920FB60F9211248A
:1000B0008F939F93AF93BF93809180019091810123
:1000C000A0918201B09183010196A11DB11D809381
:1000D000800190938101A0938201B093830181EE0E
:1000E00086BDBF91AF919F918F910F900FBE0F90E2
:1000F0001F901895F89420918001309181014091D2
:100100008201509183017894B901CA01089514BC09
:1001100083E085BD81EE86BD81E080936E0078949A
:1001200008952F923F924F925F926F927F928F929B
:100130009F92AF92BF92CF92DF92EF92FF920F9376
:100140001F93DF93CF93CDB7DEB7C75ED0400FB616
:10015000F894DEBF0FBECDBF5298539A84B18F631F
:1001600084B98AB1806C8AB987B1837C87B987B139
:10017000807C87B988B1807C88B980E880937A00D8
:1001800080E280937C0080917A00876080937A007F
:1001900080917A00806480937A0014BC83E085BDEE
:1001A00081EE86BD81E080936E007894C153DF4F6D
:1001B0001882CF5CD040C253DF4F1882CE5CD04053
:1001C000C353DF4F1882CD5CD040C753DF4F188236
:1001D00019821A821B82C95CD040CB53DF4F188230
:1001E00019821A821B82C55CD040CF53DF4F188220
:1001F00019821A821B82C15CD040C354DF4F18821F
:1002000019821A821B82CD5BD040C754DF4F1882FF
:1002100019821A821B82C95BD040CB54DF4F1882EF
:1002200019821A821B82C55BD040CF54DF4F1882DF
:1002300019821A821B82C15BD040C355DF4F1882DE
:1002400019821A821B82CD5AD040C455DF4F1882C2
:10025000CC5AD040C555DF4F1882CB5AD040C65536
:10026000DF4F1882CA5AD040C755DF4F1882C95A8B
:10027000D040C855DF4F1882C85AD040C955DF4F0B
:100280001882C75AD040CA55DF4F1882C65AD0408C
:10029000CB55DF4F1882C55AD040CC55DF4F18825E
:1002A000C45AD040CD55DF4F1882C35AD040CE55E6
:1002B000DF4F1882C25AD040CF55DF4F1882C15A43
:1002C000D040C056DF4F1882C05AD040C156DF4FD1
:1002D0001882CF59D040C256DF4F1882CE59D04035
:1002E000C356DF4F1882CD59D040C456DF4F188215
:1002F000CC59D040C556DF4F1882CB59D040C65696
:10030000DF4F1882CA59D040C756DF4F1882C959EB
:10031000D040CB56DF4F188219821A821B82C559F2
:10032000D040CF56DF4F188219821A821B82C159E2
:10033000D040C357DF4F188219821A821B82CD58D2
:10034000D040C757DF4F188219821A821B82C958C2
:10035000D040CB57DF4F188219821A821B82C558B2
:10036000D040CF57DF4F188219821A821B82C158A2
:10037000D040C358DF4F188219821A821B82CD5792
:10038000D040ED961CAE1DAE1EAE1FAEED9700EA3E
:1003900011E420E030E0E9960CAF1DAF2EAF3FAF87
:1003A000E997E5961CAE1DAE1EAE1FAEE59720ED9B
:1003B00030E240E050E0E1962CAF3DAF4EAF5FAF92
:1003C000E19788E690E1A0E0B0E0AD968CAF9DAFFC
:1003D000AEAFBFAFAD9700EF1AE020E030E0A996D6
:1003E0000CAF1DAF2EAF3FAFA99728E938E040E032
:1003F00050E0A5962CAF3DAF4EAF5FAFA59780E91B
:1004000096E0A0E0B0E0A1968CAF9DAFAEAFBFAFDD
:10041000A19708E715E020E030E06D960CAF1DAF26
:100420002EAF3FAF6D972AE134E040E050E069968F
:100430002CAF3DAF4EAF5FAF699741E050E065969E
:100440005FAF4EAF659763961CAE1DAE1EAE1FAE7E
:1004500063972F961CAE1DAE1EAE1FAE2F972B9628
:100460001FAE2B975FEF2A965FAF2A9729965FAF53
:10047000299728961FAE289727961FAE279726966E
:100480001FAE269725961FAE259724961CAE1DAE4F
:100490001EAE1FAE24971CAE1DAE1EAE1FAE18AE14
:1004A00019AE1AAE1BAE1CAA1DAA1EAA1FAA18AA14
:1004B00019AA1AAA1BAA1CA61DA61EA61FA618A624
:1004C00019A61AA61BA61CA21DA21EA21FA218A234
:1004D00019A21AA21BA21C8E1D8E1E8E1F8E1B8E91
:1004E0001A8E198E188E1F8A1E8A1D8A5B8B5A8B54
:1004F000198A2F968CAD9DADAEADBFAD2F970196ED
:10050000A11DB11D2F968CAF9DAFAEAFBFAF2F9782
:1005100085369105A105B1050CF4E1C580917A00FD
:1005200084FFFCCF80917A00806180937A00809173
:1005300079009989943021F42A968FAF2A971BC0AD
:10054000A989AA2321F427968FAF279714C0B989C8
:10055000B33021F428968FAF28970DC0E989E13098
:1005600021F42B968FAF2B9706C0F989F23019F43E
:1005700026968FAF26972A960FAD2A97E02FF0E0A8
:10058000013868F02FEF30E02E1B3F0BF901E050EF
:10059000FF4F3081309529963FAF299706C0E05034
:1005A000FF4F408129964FAF299780917A00806450
:1005B00080937A0059895F5F598B563008F0198A09
:1005C0008989806280937C008989843039F02F96F4
:1005D0001CAE1DAE1EAE1FAE2F9781C52B969FADD4
:1005E0002B979295969597709C8B4D9903C061E0DF
:1005F00070E002C064E070E0AA89A73061F4BC89B1
:10060000EB89BE1741F465960EAD1FAD6597601777
:10061000710709F46DC02C892F5F5C895E5F57708C
:100620005F5F4C894D5F47704F5F3C893C5F37701F
:100630003F5F9C899B5F97709F5F8C89895F877004
:100640008F5F269F102D1124C455DF4F1883CC5A7D
:10065000D04027702F5F269F202D1124C555DF4FD6
:100660002883CB5AD040569F202D1124C655DF4FEA
:100670002883CA5AD040469FA02D1124C755DF4F6A
:10068000A883C95AD040369FB02D1124C855DF4FDA
:10069000B883C85AD040969FE02D1124C955DF4F2A
:1006A000E883C75AD040869FF02D1124CA55DF4FEA
:1006B000F883C65AD040CB55DF4F5883C55AD04037
:1006C000CC55DF4F4883C45AD040CD55DF4F3883D7
:1006D000C35AD040CE55DF4F9883C25AD040CF5531
:1006E000DF4F8883C15AD04065967FAF6EAF659764
:1006F00028960FAD2897063070F4E996ECACFDAC67
:100700000EAD1FADE99755E015950795F794E79461
:100710005A95D1F7FDC128961FAD28971A3038F4A5
:10072000E996ECACFDAC0EAD1FADE997EAC1289699
:100730002FAD2897203170F4E996ECACFDAC0EADEE
:100740001FADE99746E015950795F794E7944A950C
:10075000D1F712C028963FAD28973631F8F4E996C4
:10076000ECACFDAC0EAD1FADE99735E015950795E6
:10077000F794E7943A95D1F7E9968CAD9DADAEAD7F
:10078000BFADE99724E0B595A795979587952A95EC
:10079000D1F7E80EF91E0A1F1B1FBAC128964FADEC
:1007A00028974C3160F5E996ECACFDAC0EAD1FAD71
:1007B000E997A5E015950795F794E794AA95D1F7E1
:1007C000E9968CAD9DADAEADBFADE997F4E0B595C2
:1007D000A79597958795FA95D1F7E80EF91E0A1F08
:1007E0001B1FE9968CAD9DADAEADBFADE997E6E0C0
:1007F000B595A79597958795EA95D1F7CACF28968D
:100800005FAD2897503238F4E996ECACFDAC0EADF4
:100810001FADE99757C128968FAD2897803470F4A3
:10082000E996ECACFDAC0EAD1FADE99775E0159502
:100830000795F794E7947A95D1F712C028969FAD63
:1008400028979035D8F4E996ECACFDAC0EAD1FAD11
:10085000E99764E015950795F794E7946A95D1F7C1
:10086000E9968CAD9DADAEADBFADE99753E0B595C2
:10087000A795979587955A95D1F78BCF2896AFADC9
:100880002897A03660F5E996ECACFDAC0EAD1FAD37
:10089000E99744E015950795F794E7944A95D1F7C1
:1008A000E9968CAD9DADAEADBFADE99733E0B595A2
:1008B000A795979587953A95D1F7E80EF91E0A1FE7
:1008C0001B1FE9968CAD9DADAEADBFADE99725E0A0
:1008D000B595A795979587952A95D1F75ACF2896DC
:1008E000BFAD2897B03738F4E996ECACFDAC0EAD4F
:1008F0001FADE997C3C02896EFAD2897E7FD0EC05E
:10090000E996ECACFDAC0EAD1FADE997B4E01595E2
:100910000795F794E794BA95D1F712C02896FFADE2
:100920002897FE38D8F4E996ECACFDAC0EAD1FADBF
:10093000E997A3E015950795F794E794AA95D1F761
:10094000E9968CAD9DADAEADBFADE997F2E0B59542
:10095000A79597958795FA95D1F71BCF28960FAD58
:100960002897003AF8F4E996ECACFDAC0EAD1FAD5B
:10097000E997E3E015950795F794E794EA95D1F7A1
:10098000E9968CAD9DADAEADBFADE99772E0B59582
:10099000A795979587957A95D1F7E80EF91E0A1FC6
:1009A0001B1FEACE28961FAD2897123B58F4E996F4
:1009B000ECACFDAC0EAD1FADE99715950795F7941E
:1009C000E794A6C028962FAD2897243B70F4E996AB
:1009D000ECACFDAC0EAD1FADE99754E01595079555
:1009E000F794E7945A95D1F725C028963FAD2897FC
:1009F0003C3B70F4E996ECACFDAC0EAD1FADE99755
:100A000043E015950795F794E7944A95D1F712C0FE
:100A100028964FAD2897443CC0F4E996ECACFDAC69
:100A20000EAD1FADE99732E015950795F794E79461
:100A30003A95D1F7E9968CAD9DADAEADBFADE997D6
:100A4000B595A79597958795A4CE28965FAD2897DD
:100A50005A3CE0F4E996ECACFDAC0EAD1FADE99765
:100A6000EE0CFF1C001F111FE9968CAD9DADAEADC5
:100A7000BFADE997E80EF91E0A1F1B1F82E015950E
:100A80000795F794E7948A95D1F742C028969FADD1
:100A900028979E3CF8F4E996ECACFDAC0EAD1FAD8A
:100AA000E997B3E0EE0CFF1C001F111FBA95D1F7B8
:100AB000E9962CAD3DAD4EAD5FADE997E21AF30A74
:100AC000040B150BA3E015950795F794E794AA95E9
:100AD000D1F71EC0E996ECACFDAC0EAD1FADE997A9
:100AE000F4E0EE0CFF1C001F111FFA95D1F7E996F8
:100AF0008CAD9DADAEADBFADE997E81AF90A0A0B12
:100B00001B0BE4E015950795F794E794EA95D1F768
:100B1000C455DF4F3881CC5AD040232F30E040E01D
:100B200050E0C452DF4F288339834A835B83CC5D16
:100B3000D040C801B7010E94E615C901DA01E1966B
:100B40008CAF9DAFAEAFBFAFE1970A97A105B105DE
:100B500054F48AE090E0A0E0B0E0E1968CAF9DAF65
:100B6000AEAFBFAFE197C555DF4F3881CB5AD0400C
:100B7000232F30E040E050E0C852DF4F2883398314
:100B80004A835B83C85DD040C801B7010E94E61567
:100B9000C901DA01AD968CAF9DAFAEAFBFAFAD97D7
:100BA0000A97A105B10554F48AE090E0A0E0B0E016
:100BB000AD968CAF9DAFAEAFBFAFAD97C655DF4F13
:100BC0003881CA5AD040232F30E040E050E0CC5268
:100BD000DF4F288339834A835B83C45DD040C801DB
:100BE000B7010E94E615C901DA01A9968CAF9DAF45
:100BF000AEAFBFAFA9970A97A105B10554F48AE03B
:100C000090E0A0E0B0E0A9968CAF9DAFAEAFBFAFD3
:100C1000A997C755DF4F3881C95AD040232F30E0FC
:100C200040E050E0C053DF4F288339834A835B8321
:100C3000C05DD040C801B7010E94E615C901DA01C4
:100C4000A5968CAF9DAFAEAFBFAFA5970A97A10594
:100C5000B10554F48AE090E0A0E0B0E0A5968CAF36
:100C60009DAFAEAFBFAFA597C855DF4F9881C85AAB
:100C7000D040292E332444245524C801B701A201B1
:100C800091010E94E615C901DA01A1968CAF9DAFD2
:100C9000AEAFBFAFA1970A97A105B10554F42AE002
:100CA00030E040E050E0A1962CAF3DAF4EAF5FAFDB
:100CB000A197C955DF4F3881C75AD040632E77249A
:100CC00088249924C801B701A40193010E94E61564
:100CD000C901DA016D968CAF9DAFAEAFBFAF6D9716
:100CE0000A97A105B10554F48AE090E0A0E0B0E0D5
:100CF0006D968CAF9DAFAEAFBFAF6D97CA55DF4F4E
:100D00009881C65AD040A92EBB24CC24DD24C8012A
:100D1000B701A60195010E94E615C901DA0169969D
:100D20008CAF9DAFAEAFBFAF69970A97A105B10574
:100D300054F40AE010E020E030E069960CAF1DAFFB
:100D40002EAF3FAF6997E9966CAD7DAD8EAD9FAD8F
:100D5000E997CC52DF4F288139814A815B81C45D9C
:100D6000D0400E94E615C052DF4F2883C05ED040BD
:100D7000CF51DF4F3883C15ED040CE51DF4F488323
:100D8000C25ED040CD51DF4F5883C35ED040C052C9
:100D9000DF4F288139814A815B81C05ED040C357D3
:100DA000DF4F288339834A835B83CD58D040E9964F
:100DB0006CAD7DAD8EAD9FADE997C053DF4F2881FF
:100DC00039814A815B81C05DD0400E94E615CC51DB
:100DD000DF4F2883C45ED040CB51DF4F3883C55EE0
:100DE000D040CA51DF4F4883C65ED040C951DF4F63
:100DF0005883C75ED040CC51DF4F88819981AA814A
:100E0000BB81C45ED040C757DF4F88839983AA83D4
:100E1000BB83C958D040E9966CAD7DAD8EAD9FAD1A
:100E2000E997A20191010E94E61519012A01CB5709
:100E3000DF4F288239824A825B82C558D040E996CA
:100E40006CAD7DAD8EAD9FADE997A40193010E947D
:100E5000E61539014A01CF57DF4F688279828A82CD
:100E60009B82C158D040E9966CAD7DAD8EAD9FADF3
:100E7000E997A60195010E94E61559016A01C35838
:100E8000DF4FA882B982CA82DB82CD57D040279635
:100E90009FAD279797FD02C01D8A06C02796AFAD6C
:100EA0002797A370AE5FAD8BE9966CAD7DAD8EAD2F
:100EB0009FADE997C452DF4F288139814A815B8118
:100EC000CC5DD0400E94E615C901DA01CB56DF4F58
:100ED00088839983AA83BB83C559D040E9966CADBA
:100EE0007DAD8EAD9FADE997C852DF4F2881398126
:100EF0004A815B81C85DD0400E94E615C901DA01D4
:100F0000CF56DF4F88839983AA83BB83C159D040D2
:100F10002796BFAD27972B2F30E02F773070C90170
:100F2000880F991F880F991F820F931F880F892F91
:100F3000881F990BE82FEE5FEE8B2696FFAD269764
:100F4000EF2EFF2400E010E0C052DF4F28813981EE
:100F50004A815B81C05ED0402A50304040405040C2
:100F6000A9968CAD9DADAEADBFADA997281B390B31
:100F70004A0B5B0BC052DF4F288339834A835B8364
:100F8000C05ED040CA01B901A80197010E94C715EF
:100F9000272F382F492F552747FD5A952CA73DA7B6
:100FA0004EA75FA7CC51DF4F88819981AA81BB8171
:100FB000C45ED0400A97A109B109A5962CAD3DADFC
:100FC0004EAD5FADA597821B930BA40BB50BCC5117
:100FD000DF4F88839983AA83BB83C45ED040BC0162
:100FE000CD01A80197010E94C715272F382F492F3F
:100FF000552747FD5A9528A739A74AA75BA786EF2B
:101000009FEFAFEFBFEF280E391E4A1E5B1EA19661
:101010002CAD3DAD4EAD5FADA197221A330A440A07
:10102000550AC201B101A80197010E94C715272FD7
:10103000382F492F552747FD5A952CA33DA34EA382
:101040005FA386EF9FEFAFEFBFEF680E791E8A1E9A
:101050009B1E6D962CAD3DAD4EAD5FAD6D97621A8A
:10106000730A840A950AC401B301A80197010E947A
:10107000C715272F382F492F552747FD5A9528A3E5
:1010800039A34AA35BA386EF9FEFAFEFBFEFA80E94
:10109000B91ECA1EDB1E69962CAD3DAD4EAD5FADCF
:1010A0006997A21AB30AC40AD50AC601B501A801F4
:1010B00097010E94C715072F182F292F332727FDC7
:1010C0003A950C8F1D8F2E8F3F8F1C891B8B2F966F
:1010D0001CAE1DAE1EAE1FAE2F9727E02A8B349993
:1010E00004C025961FAE25971EC125963FAD2597B6
:1010F000332329F041E025964FAF259714C1ED9693
:101100008CAD9DADAEADBFADED97CB56DF4F088139
:1011100019812A813B81C559D040801B910BA20BBC
:10112000B30BC753DF4F88839983AA83BB83C95C02
:10113000D040ED962CAD3DAD4EAD5FADED97CF56A9
:10114000DF4F88819981AA81BB81C159D040281B7A
:10115000390B4A0B5B0BCB53DF4F288339834A8310
:101160005B83C55CD040ED960CAD1DAD2EAD3FADA3
:10117000ED97C357DF4F88819981AA81BB81CD58F4
:10118000D040081B190B2A0B3B0B24968CAD9DAD50
:10119000AEADBFAD2497081B190B2A0B3B0BCF53E9
:1011A000DF4F088319832A833B83C15CD040ED96CF
:1011B0000CAD1DAD2EAD3FADED97C757DF4F88810C
:1011C0009981AA81BB81C958D040081B190B2A0BF1
:1011D0003B0B8CAD9DADAEADBFAD081B190B2A0B03
:1011E0003B0BC354DF4F088319832A833B83CD5BBA
:1011F000D040ED960CAD1DAD2EAD3FADED97CB576C
:10120000DF4F88819981AA81BB81C558D040081BD6
:10121000190B2A0B3B0B88AD99ADAAADBBAD081BD2
:10122000190B2A0B3B0BC754DF4F088319832A8302
:101230003B83C95BD040ED960CAD1DAD2EAD3FADEF
:10124000ED97CF57DF4F88819981AA81BB81C15823
:10125000D040081B190B2A0B3B0B8CA99DA9AEA9EA
:10126000BFA9081B190B2A0B3B0BCB54DF4F08837C
:1012700019832A833B83C55BD040ED960CAD1DAD31
:101280002EAD3FADED97C358DF4F88819981AA817C
:10129000BB81CD57D040081B190B2A0B3B0BC35504
:1012A000DF4F088319832A833B83CD5AD04088A916
:1012B00099A9AAA9BBA9081B190B2A0B3B0BCF5450
:1012C000DF4F088319832A833B83C15BD040C0561C
:1012D000DF4F1882C05AD040C156DF4F1882CF5915
:1012E000D040C256DF4F1882CE59D040C356DF4F90
:1012F0001882CD59D040C456DF4F1882CC59D04007
:10130000C556DF4F1882CB59D040C656DF4F1882E2
:10131000CA59D040C756DF4F1882C959D04091E012
:1013200025969FAF2597F894009180011091810137
:101330002091820130918301ED960CAF1DAF2EAF4D
:101340003FAFED9778944A9B43C5C153DF4F188157
:10135000CF5CD040112309F0A7C6C253DF4F2881CC
:10136000CE5CD0402A3030F42F5FC253DF4F288349
:10137000CE5CD040C253DF4F3881CE5CD0403A3093
:1013800009F092C6CA55DF4F4881C65AD040415035
:10139000C656DF4F4883CA59D0405B98ED968CAD56
:1013A0009DADAEADBFADED97E5960CAD1DAD2EADCF
:1013B0003FADE597801B910BA20BB30BE9968CAF69
:1013C0009DAFAEAFBFAFE99728961FAD28971630F7
:1013D00050F47C018D01B5E015950795F794E794DD
:1013E000BA95D1F7FDC128962FAD28972A3038F449
:1013F000E996ECACFDAC0EAD1FADE997EAC12896BD
:101400003FAD2897303170F4E996ECACFDAC0EADF1
:101410001FADE997A6E015950795F794E794AA956F
:10142000D1F712C028964FAD28974631F8F4E996C7
:10143000ECACFDAC0EAD1FADE997F5E01595079549
:10144000F794E794FA95D1F7E9968CAD9DADAEADE2
:10145000BFADE997E4E0B595A79597958795EA958F
:10146000D1F7E80EF91E0A1F1B1FBAC128965FADFF
:1014700028975C3160F5E996ECACFDAC0EAD1FAD84
:10148000E99775E015950795F794E7947A95D1F764
:10149000E9968CAD9DADAEADBFADE99764E0B59575
:1014A000A795979587956A95D1F7E80EF91E0A1FBB
:1014B0001B1FE9968CAD9DADAEADBFADE99756E073
:1014C000B595A795979587955A95D1F7CACF289640
:1014D0008FAD2897803238F4E996ECACFDAC0EADB8
:1014E0001FADE99757C128969FAD2897903470F4A7
:1014F000E996ECACFDAC0EAD1FADE99745E0159556
:101500000795F794E7944A95D1F712C02896AFADA6
:101510002897A035D8F4E996ECACFDAC0EAD1FAD24
:10152000E99734E015950795F794E7943A95D1F744
:10153000E9968CAD9DADAEADBFADE99723E0B59515
:10154000A795979587952A95D1F78BCF2896BFAD0C
:101550002897B03660F5E996ECACFDAC0EAD1FAD4A
:10156000E997F4E015950795F794E794FA95D1F784
:10157000E9968CAD9DADAEADBFADE997E3E0B59515
:10158000A79597958795EA95D1F7E80EF91E0A1F5A
:101590001B1FE9968CAD9DADAEADBFADE99775E073
:1015A000B595A795979587957A95D1F75ACF2896AF
:1015B000EFAD2897E03738F4E996ECACFDAC0EAD12
:1015C0001FADE997C3C02896FFAD2897F7FD0EC061
:1015D000E996ECACFDAC0EAD1FADE99764E0159556
:1015E0000795F794E7946A95D1F712C028960FAD46
:1015F00028970E38D8F4E996ECACFDAC0EAD1FADD3
:10160000E99753E015950795F794E7945A95D1F724
:10161000E9968CAD9DADAEADBFADE99742E0B59515
:10162000A795979587954A95D1F71BCF28961FAD1B
:101630002897103AF8F4E996ECACFDAC0EAD1FAD6E
:10164000E99733E015950795F794E7943A95D1F724
:10165000E9968CAD9DADAEADBFADE99722E0B595F5
:10166000A795979587952A95D1F7E80EF91E0A1F39
:101670001B1FEACE28962FAD2897223B58F4E996F7
:10168000ECACFDAC0EAD1FADE99715950795F79441
:10169000E794A6C028963FAD2897343B70F4E996AE
:1016A000ECACFDAC0EAD1FADE997F4E015950795D8
:1016B000F794E794FA95D1F725C028964FAD28976F
:1016C0004C3B70F4E996ECACFDAC0EAD1FADE99768
:1016D000E3E015950795F794E794EA95D1F712C0E2
:1016E00028965FAD2897543CC0F4E996ECACFDAC6D
:1016F0000EAD1FADE99772E015950795F794E79445
:101700007A95D1F7E9968CAD9DADAEADBFADE997B9
:10171000B595A79597958795A4CE28968FAD2897D0
:101720008A3CE0F4E996ECACFDAC0EAD1FADE99758
:10173000EE0CFF1C001F111FE9962CAD3DAD4EAD08
:101740005FADE997E20EF31E041F151F42E01595E9
:101750000795F794E7944A95D1F742C028963FAD94
:1017600028973E3CF8F4E996ECACFDAC0EAD1FAD0D
:10177000E99733E0EE0CFF1C001F111F3A95D1F7DB
:10178000E9968CAD9DADAEADBFADE997E81AF90A0B
:101790000A0B1B0B23E015950795F794E7942A9500
:1017A000D1F71EC0E996ECACFDAC0EAD1FADE997CC
:1017B00094E0EE0CFF1C001F111F9A95D1F7E996DB
:1017C0002CAD3DAD4EAD5FADE997E21AF30A040BC7
:1017D000150B84E015950795F794E7948A95D1F752
:1017E000C455DF4F9881CC5AD040892F90E0A0E0BB
:1017F000B0E08D879E87AF87B88BC801B7012D8574
:101800003E854F8558890E94E615C901DA01E196A7
:101810008CAF9DAFAEAFBFAFE1970A97A105B10501
:1018200054F42AE030E040E050E0E1962CAF3DAFC8
:101830004EAF5FAFE197C555DF4F9881CB5AD0408F
:10184000892F90E0A0E0B0E089879A87AB87BC87BA
:10185000C801B70129853A854B855C850E94E6154C
:10186000C901DA01AD968CAF9DAFAEAFBFAFAD97FA
:101870000A97A105B10554F42AE030E040E050E0B9
:10188000AD962CAF3DAF4EAF5FAFAD97C655DF4FB6
:101890009881CA5AD040892F90E0A0E0B0E08D83B3
:1018A0009E83AF83B887C801B7012D813E814F81E8
:1018B00058850E94E615C901DA01A9968CAF9DAF43
:1018C000AEAFBFAFA9970A97A105B10554F42AE0BE
:1018D00030E040E050E0A9962CAF3DAF4EAF5FAF97
:1018E000A997C755DF4F9881C95AD040892F90E0FA
:1018F000A0E0B0E089839A83AB83BC83C801B701C1
:1019000029813A814B815C810E94E615C901DA0187
:10191000A5968CAF9DAFAEAFBFAFA5970A97A105B7
:10192000B10554F42AE030E040E050E0A5962CAF39
:101930003DAF4EAF5FAFA597C855DF4F3881C85A4E
:10194000D040232E332444245524C801B701A201DA
:1019500091010E94E615C901DA01A1968CAF9DAFF5
:10196000AEAFBFAFA1970A97A105B10554F48AE0C5
:1019700090E0A0E0B0E0A1968CAF9DAFAEAFBFAF5E
:10198000A197C955DF4F9881C75AD040692E772457
:1019900088249924C801B701A40193010E94E61587
:1019A000C901DA016D968CAF9DAFAEAFBFAF6D9739
:1019B0000A97A105B10554F42AE030E040E050E078
:1019C0006D962CAF3DAF4EAF5FAF6D97CA55DF4FF1
:1019D0003881C65AD040A32EBB24CC24DD24C801B4
:1019E000B701A60195010E94E615C901DA016996C1
:1019F0008CAF9DAFAEAFBFAF69970A97A105B10598
:101A000054F48AE090E0A0E0B0E069968CAF9DAF1E
:101A1000AEAFBFAF6997C455DF4F9881CC5AD04065
:101A20009150C056DF4F9883C05AD040C555DF4F04
:101A3000A881CB5AD040A150C156DF4FA883CF59BF
:101A4000D040C655DF4FB881CA5AD040B150C256B7
:101A5000DF4FB883CE59D040C755DF4FE881C95A10
:101A6000D040E150C356DF4FE883CD59D040C85530
:101A7000DF4FF881C85AD040F150C456DF4FF88389
:101A8000CC59D040C955DF4F0881C75AD0400150CA
:101A9000C556DF4F0883CB59D040E9966CAD7DAD7C
:101AA0008EAD9FADE9972D853E854F8558890E9463
:101AB000E615C901DA01CB56DF4F88839983AA83E3
:101AC000BB83C559D040E9966CAD7DAD8EAD9FAD61
:101AD000E99729853A854B855C850E94E615C90101
:101AE000DA01CF56DF4F88839983AA83BB83C1591C
:101AF000D040E9966CAD7DAD8EAD9FADE9972D815F
:101B00003E814F8158850E94E615C901DA01C3570D
:101B1000DF4F88839983AA83BB83CD58D040E99651
:101B20006CAD7DAD8EAD9FADE99729813A814B813A
:101B30005C810E94E615C901DA01C757DF4F88832F
:101B40009983AA83BB83C958D040E9966CAD7DAD1B
:101B50008EAD9FADE997A20191010E94E615C901E2
:101B6000DA01CB57DF4F88839983AA83BB83C5589B
:101B7000D040E9966CAD7DAD8EAD9FADE997A401E7
:101B800093010E94E615C901DA01CF57DF4F888320
:101B90009983AA83BB83C158D040E9966CAD7DADD3
:101BA0008EAD9FADE997A60195010E94E615C9018A
:101BB000DA01C358DF4F88839983AA83BB83CD574B
:101BC000D040ED962CAD3DAD4EAD5FADED97CB5613
:101BD000DF4F88819981AA81BB81C559D040281BDC
:101BE000390B4A0B5B0BC753DF4F288339834A837A
:101BF0005B83C95CD040ED960CAD1DAD2EAD3FAD05
:101C0000ED97CF56DF4F88819981AA81BB81C15959
:101C1000D040081B190B2A0B3B0BCB53DF4F08831B
:101C200019832A833B83C55CD040ED960CAD1DAD76
:101C30002EAD3FADED97C357DF4F88819981AA81C3
:101C4000BB81CD58D040081B190B2A0B3B0B2496A7
:101C50008CAD9DADAEADBFAD2497081B190B2A0B03
:101C60003B0BCF53DF4F088319832A833B83C15C2F
:101C7000D040ED960CAD1DAD2EAD3FADED97C757E5
:101C8000DF4F88819981AA81BB81C958D040081B48
:101C9000190B2A0B3B0B8CAD9DADAEADBFAD081B38
:101CA000190B2A0B3B0BC354DF4F088319832A837C
:101CB0003B83CD5BD040ED960CAD1DAD2EAD3FAD61
:101CC000ED97CB57DF4F88819981AA81BB81C55899
:101CD000D040081B190B2A0B3B0B88AD99ADAAAD60
:101CE000BBAD081B190B2A0B3B0BC754DF4F0883F6
:101CF00019832A833B83C95BD040ED960CAD1DADA3
:101D00002EAD3FADED97CF57DF4F88819981AA81E6
:101D1000BB81C158D040081B190B2A0B3B0B8CA967
:101D20009DA9AEA9BFA9081B190B2A0B3B0BCB54CD
:101D3000DF4F088319832A833B83C55BD040ED9630
:101D40000CAD1DAD2EAD3FADED97C358DF4F888173
:101D50009981AA81BB81CD57D040081B190B2A0B52
:101D60003B0BC355DF4F088319832A833B83CD5A2E
:101D7000D04088A999A9AAA9BBA9081B190B2A0BAD
:101D80003B0BCF54DF4F088319832A833B83C15B0E
:101D9000D040C656DF4F9881CA59D040C756DF4F52
:101DA0009883C959D040ED960CAD1DAD2EAD3FAD19
:101DB000ED97E5960CAF1DAF2EAF3FAFE597B9019C
:101DC000A80111E0C153DF4F1883CF5CD04072C12E
:101DD000C353DF4F2881CD5CD0402A3030F42F5FD1
:101DE000C353DF4F2883CD5CD040C353DF4F3881CE
:101DF000CD5CD0403A3039F063964CAD5DAD6EAD00
:101E00007FAD63974BC15B9A63964CAD5DAD6EAD94
:101E10007FAD6397E9968CAD9DADAEADBFADE99753
:101E2000480F591F6A1F7B1FED960CAD1DAD2EADDF
:101E30003FADED9704171507260737073CF4639667
:101E40004CAD5DAD6EAD7FAD639723C1C455DF4F23
:101E50001881CC5AD0401150C056DF4F1883C05A59
:101E6000D040C555DF4F2881CB5AD0402150C156B4
:101E7000DF4F2883CF59D040C655DF4F3881CA5A2B
:101E8000D0403150C256DF4F3883CE59D040C7556D
:101E9000DF4F8881C95AD0408150C356DF4F8883B5
:101EA000CD59D040C855DF4F9881C85AD040915085
:101EB000C456DF4F9883CC59D040C955DF4FA88115
:101EC000C75AD040A150C556DF4FA883CB59D04048
:101ED000CA55DF4FB881C65AD040B150C656DF4F01
:101EE000B883CA59D0408A019B01CB56DF4F888105
:101EF0009981AA81BB81C559D040081B190B2A0BB7
:101F00003B0BC753DF4F088319832A833B83C95C8C
:101F1000D0408A019B01CF56DF4F88819981AA81E9
:101F2000BB81C159D040081B190B2A0B3B0BCB536B
:101F3000DF4F088319832A833B83C55CD0408A0125
:101F40009B01C357DF4F88819981AA81BB81CD58FE
:101F5000D040081B190B2A0B3B0B24968CAD9DAD72
:101F6000AEADBFAD2497081B190B2A0B3B0BCF530B
:101F7000DF4F088319832A833B83C15CD0408A01E9
:101F80009B01C757DF4F88819981AA81BB81C958BE
:101F9000D040081B190B2A0B3B0B8CAD9DADAEAD91
:101FA000BFAD081B190B2A0B3B0BC354DF4F088333
:101FB00019832A833B83CD5BD0408A019B01CB5799
:101FC000DF4F88819981AA81BB81C558D040081B09
:101FD000190B2A0B3B0B88AD99ADAAADBBAD081B05
:101FE000190B2A0B3B0BC754DF4F088319832A8335
:101FF0003B83C95BD0408A019B01CF57DF4F88816B
:102000009981AA81BB81C158D040081B190B2A0BAA
:102010003B0B8CA99DA9AEA9BFA9081B190B2A0BC4
:102020003B0BCB54DF4F088319832A833B83C55B6B
:10203000D0408A019B01C358DF4F88819981AA81D2
:10204000BB81CD57D040081B190B2A0B3B0BC35546
:10205000DF4F088319832A833B83CD5AD04088A958
:1020600099A9AAA9BBA9081B190B2A0B3B0BCF5492
:10207000DF4F088319832A833B83C15BD040C65658
:10208000DF4F9881CA59D040C756DF4F9883C9594E
:10209000D040C153DF4F1882CF5CD040C253DF4FD6
:1020A0001882CE5CD0400BC063964CAD5DAD6EAD7A
:1020B0007FAD6397C353DF4F1882CD5CD040CB56C2
:1020C000DF4F88819981AA81BB81C559D040C75310
:1020D000DF4F088119812A813B81C95CD040800F84
:1020E000911FA21FB31FED960CAD1DAD2EAD3FADE0
:1020F000ED97081719072A073B0784F14C9B28988E
:10210000C056DF4F1881C05AD0401F5FC056DF4F06
:102110001883C05AD040C455DF4F2881CC5AD040D4
:10212000121778F4ED968CAD9DADAEADBFADED97C9
:10213000C753DF4F88839983AA83BB83C95CD04090
:102140000DC0C753DF4F488359836A837B83C95CC3
:10215000D040C056DF4F1882C05AD040CF56DF4F14
:1021600088819981AA81BB81C159D040CB53DF4F6F
:10217000088119812A813B81C55CD040800F911F65
:10218000A21FB31FED960CAD1DAD2EAD3FADED976B
:10219000081719072A073B0784F14C9B2998C15659
:1021A000DF4F1881CF59D0401F5FC156DF4F1883D2
:1021B000CF59D040C555DF4F2881CB5AD040121798
:1021C00078F4ED968CAD9DADAEADBFADED97CB5334
:1021D000DF4F88839983AA83BB83C55CD0400DC041
:1021E000CB53DF4F488359836A837B83C55CD040E0
:1021F000C156DF4F1882CF59D040CF53DF4F88816F
:102200009981AA81BB81C15CD040C357DF4F08814F
:1022100019812A813B81CD58D040800F911FA21F88
:10222000B31F24960CAD1DAD2EAD3FAD2497800F8E
:10223000911FA21FB31FED960CAD1DAD2EAD3FAD8E
:10224000ED97081719072A073B070CF491C0299648
:102250001FAD2997812F90E028E030E0CB55DF4F6C
:10226000A881C55AD0402A1B310902C0959587958F
:102270002A95E2F7C256DF4F0880CE59D04002C0FF
:10228000959587950A94E2F780FF02C04C9B2A98A7
:10229000C256DF4FB881CE59D040BF5FC256DF4F24
:1022A000B883CE59D040CB55DF4FE881C55AD040D6
:1022B000BE1778F4ED960CAD1DAD2EAD3FADED978C
:1022C000CF53DF4F088319832A833B83C15CD040FF
:1022D0000EC0CF53DF4F488359836A837B83C15C31
:1022E000D040C256DF4F1882CE59D0401B8E1E8977
:1022F000123028F41CAE1DAE1EAE1FAE39C024969F
:102300008CAD9DADAEADBFAD2497181619061A065B
:102310001B063CF024961CAE1DAE1EAE1FAE2497CD
:1023200013C024960CAD1DAD2EAD3FAD2497309556
:102330002095109501951F4F2F4F3F4F24960CAFBE
:102340001DAF2EAF3FAF24971B8D112351F48CA5E9
:102350009DA5AEA5BFA524968CAF9DAFAEAFBFAF78
:1023600024979B8D9F5F9B8FAE899A1708F01B8ED9
:10237000C757DF4F88819981AA81BB81C958D04056
:10238000C354DF4F088119812A813B81CD5BD04046
:10239000800F911FA21FB31F0CAD1DAD2EAD3FAD21
:1023A000800F911FA21FB31FED960CAD1DAD2EAD7A
:1023B0003FADED97081719072A073B070CF487C0B4
:1023C00029961FAD2997812F90E028E030E0CC5569
:1023D000DF4FA881C45AD0402A1B310902C095950D
:1023E00087952A95E2F7C356DF4F0880CD59D04034
:1023F00002C0959587950A94E2F780FF02C04C9B36
:102400002B98C356DF4FB881CD59D040BF5FC3561C
:10241000DF4FB883CD59D040CC55DF4FE881C45A47
:10242000D040BE1778F4ED960CAD1DAD2EAD3FAD8E
:10243000ED97C354DF4F088319832A833B83CD5B19
:10244000D0400EC0C354DF4F488359836A837B83D7
:10245000CD5BD040C356DF4F1882CD59D0401A8E85
:102460001E89123028F41CAE1DAE1EAE1FAE2FC04A
:102470008CAD9DADAEADBFAD181619061A061B0684
:102480002CF01CAE1DAE1EAE1FAE0FC00CAD1DADB0
:102490002EAD3FAD30952095109501951F4F2F4FD4
:1024A0003F4F0CAF1DAF2EAF3FAF1A8D112341F43C
:1024B00088A599A5AAA5BBA58CAF9DAFAEAFBFAFB0
:1024C0009A8D9F5F9A8FAE899A1708F01A8EC7541B
:1024D000DF4F88819981AA81BB81C95BD040CB57EE
:1024E000DF4F088119812A813B81C558D040800F78
:1024F000911FA21FB31F08AD19AD2AAD3BAD800FD0
:10250000911FA21FB31FED960CAD1DAD2EAD3FADBB
:10251000ED97081719072A073B070CF48BC029967B
:102520001FAD2997812F90E028E030E0CD55DF4F97
:10253000A881C35AD0402A1B310902C095958795BE
:102540002A95E2F7C456DF4F0880CC59D04002C02C
:10255000959587950A94E2F780FF02C04C9B2C98D2
:10256000C456DF4FB881CC59D040BF5FC456DF4F4F
:10257000B883CC59D040CD55DF4FE881C35AD04005
:10258000BE1778F4ED960CAD1DAD2EAD3FADED97B9
:10259000C754DF4F088319832A833B83C95BD0402C
:1025A0000EC0C754DF4F488359836A837B83C95B5E
:1025B000D040C456DF4F1882CC59D040198E1E89A6
:1025C000123028F418AE19AE1AAE1BAE33C088AD67
:1025D00099ADAAADBBAD181619061A061B062CF04C
:1025E00018AE19AE1AAE1BAE13C0998DAD899A17ED
:1025F00078F008AD19AD2AAD3BAD3095209510951A
:1026000001951F4F2F4F3F4F08AF19AF2AAF3BAF78
:10261000198D112341F48CA19DA1AEA1BFA188AF5A
:1026200099AFAAAFBBAF998D9F5F998FAE899A176B
:1026300008F0198ECB54DF4F88819981AA81BB8124
:10264000C55BD040CF57DF4F088119812A813B817C
:10265000C158D040800F911FA21FB31F0CA91DA904
:102660002EA93FA9800F911FA21FB31FED960CAD9D
:102670001DAD2EAD3FADED97081719072A073B0793
:102680000CF48BC029961FAD2997812F90E028E08C
:1026900030E0CE55DF4FA881C25AD0402A1B310905
:1026A00002C0959587952A95E2F7C556DF4F0880B9
:1026B000CB59D04002C0959587950A94E2F780FFE8
:1026C00002C04C9B2D98C556DF4FB881CB59D040E6
:1026D000BF5FC556DF4FB883CB59D040CE55DF4FD3
:1026E000E881C25AD040BE1778F4ED960CAD1DAD0E
:1026F0002EAD3FADED97CB54DF4F088319832A836E
:102700003B83C55BD0400EC0CB54DF4F4883598319
:102710006A837B83C55BD040C556DF4F1882CB5997
:10272000D040188E1E89123028F41CAA1DAA1EAA99
:102730001FAA33C08CA99DA9AEA9BFA91816190656
:102740001A061B062CF01CAA1DAA1EAA1FAA13C03B
:10275000988DAD899A1778F00CA91DA92EA93FA9CB
:1027600030952095109501951F4F2F4F3F4F0CAB83
:102770001DAB2EAB3FAB188D112341F488A199A15D
:10278000AAA1BBA18CAB9DABAEABBFAB988D9F5F3D
:10279000988FAE899A1708F0188ECF54DF4F888132
:1027A0009981AA81BB81C15BD040C358DF4F0881AA
:1027B00019812A813B81CD57D040800F911FA21FE4
:1027C000B31F08A919A92AA93BA9800F911FA21F0D
:1027D000B31FED960CAD1DAD2EAD3FADED970817B7
:1027E00019072A073B070CF48BC029961FAD2997C0
:1027F000812F90E028E030E0CF55DF4FA881C15A0B
:10280000D0402A1B310902C0959587952A95E2F799
:10281000C656DF4F0880CA59D04002C095958795AB
:102820000A94E2F780FF02C04C9B5F98C656DF4FC8
:10283000B881CA59D040BF5FC656DF4FB883CA5966
:10284000D040CF55DF4FE881C15AD040BE1778F451
:10285000ED960CAD1DAD2EAD3FADED97CF54DF4FD6
:10286000088319832A833B83C15BD0400EC0CF54B9
:10287000DF4F488359836A837B83C15BD040C65650
:10288000DF4F1882CA59D0401F8A1E89123028F49F
:1028900018AA19AA1AAA1BAA33C088A999A9AAA971
:1028A000BBA9181619061A061B062CF018AA19AA95
:1028B0001AAA1BAA13C09F89AD899A1778F008A994
:1028C00019A92AA93BA930952095109501951F4F6C
:1028D0002F4F3F4F08AB19AB2AAB3BAB1F891123DE
:1028E00041F48C8D9D8DAE8DBF8D88AB99ABAAAB1D
:1028F000BBAB9F899F5F9F8BAE899A1708F01F8A99
:10290000C358DF4F88819981AA81BB81CD57D040C0
:10291000C355DF4F088119812A813B81CD5AD040B0
:10292000800F911FA21FB31FED960CAD1DAD2EADF4
:102930003FADED97081719072A073B0784F14C9B19
:102940005E98C756DF4F1881C959D0401F5FC756E0
:10295000DF4F1883C959D040CA55DF4F2881C65A66
:10296000D040121778F4ED968CAD9DADAEADBFADF5
:10297000ED97C355DF4F88839983AA83BB83CD5AD4
:10298000D0400DC0C355DF4F488359836A837B8392
:10299000CD5AD040C756DF4F1882C959D040C753CF
:1029A000DF4F88819981AA81BB81C95CD040E196C3
:1029B0000CAD1DAD2EAD3FADE197800F911FA21F55
:1029C000B31FED960CAD1DAD2EAD3FADED970817C5
:1029D00019072A073B070CF0289ACB53DF4F888151
:1029E0009981AA81BB81C55CD040AD960CAD1DAD6F
:1029F0002EAD3FADAD97800F911FA21FB31FED9677
:102A00000CAD1DAD2EAD3FADED97081719072A0788
:102A10003B070CF0299ACF53DF4F88819981AA8117
:102A2000BB81C15CD040A9960CAD1DAD2EAD3FADB4
:102A3000A997800F911FA21FB31FED960CAD1DAD7E
:102A40002EAD3FADED97081719072A073B070CF08D
:102A50002A9AC354DF4F88819981AA81BB81CD5BBB
:102A6000D040A5960CAD1DAD2EAD3FADA597800F06
:102A7000911FA21FB31FED960CAD1DAD2EAD3FAD46
:102A8000ED97081719072A073B070CF02B9AC75434
:102A9000DF4F88819981AA81BB81C95BD040A19613
:102AA0000CAD1DAD2EAD3FADA197800F911FA21FA4
:102AB000B31FED960CAD1DAD2EAD3FADED970817D4
:102AC00019072A073B070CF02C9ACB54DF4F88815B
:102AD0009981AA81BB81C55BD0406D960CAD1DADBF
:102AE0002EAD3FAD6D97800F911FA21FB31FED96C6
:102AF0000CAD1DAD2EAD3FADED97081719072A0798
:102B00003B070CF02D9ACF54DF4F88819981AA8121
:102B1000BB81C15BD04069960CAD1DAD2EAD3FAD04
:102B20006997800F911FA21FB31FED960CAD1DADCD
:102B30002EAD3FADED97081719072A073B070CF09C
:102B40005F9AC355DF4F88819981AA81BB81CD5A95
:102B5000D04069960CAD1DAD2EAD3FAD6997800F8D
:102B6000911FA21FB31FED960CAD1DAD2EAD3FAD55
:102B7000ED97081719072A073B070CF05E9A639632
:102B80004CAF5DAF6EAF7FAF63970C947902629FDD
:102B9000D001739FF001829FE00DF11D649FE00D55
:102BA000F11D929FF00D839FF00D749FF00D659FB6
:102BB000F00D9927729FB00DE11DF91F639FB00DB5
:102BC000E11DF91FBD01CF011124089597FB092EC6
:102BD00005260ED057FD04D014D00AD0001C38F4BE
:102BE00050954095309521953F4F4F4F5F4F089539
:102BF000F6F790958095709561957F4F8F4F9F4F19
:102C00000895A1E21A2EAA1BBB1BFD010DC0AA1F2D
:102C1000BB1FEE1FFF1FA217B307E407F50720F045
:102C2000A21BB30BE40BF50B661F771F881F991FC0
:102C30001A9469F760957095809590959B01AC0109
:0A2C4000BD01CF010895F894FFCF05
:102C4A00FFFEFDFBF7EFDFBF7F3F9FCFE7F3F9FC06
:102C5A00FAF5EBD7AF5F6FB7DBEDF6EEDDBB777B4F
:102C6A00BDDEBE7D7E3E5E6E767A7CBCBAB6AE9E18
:102C7A009DADB5B9D9D5CDCBD3E3C7E3F1F81F8F55
:102C8A00D3E9F4ECB367DCF0E8D8B878746C5C3C50
:102C9A003A362E1E1D1B170F1B3363C3C6CC666341
:102CAA00C6C3C5C9D1D2D46A352D5AB4AC562B4B3A
:102CBA0096A653939555AA55AA55AA55AA55AA5503
:00000001FF
